:100000000C94340018950000189500001895000015
:10001000189500001895000018950000189500002C
:10002000189500001895000018950000189500001C
:10003000189500001895000018950000189500000C
:1000400018950000189500000C94350618950000CE
:1000500018950000189500001895000018950000EC
:1000600018950000189500008FEF8DBFC0EEE6ECEC
:100070004E2E84E08EBFD4E0F4E05F2EEEEFF3E08E
:10008000A0E0B1E0A89584B7082E877F84BF88E1FF
:100090009927809360009093600088278D93319713
:1000A000E9F787E48093C40080E08093C50088E18D
:1000B0008093C1000E94750566243D983C98459A3E
:1000C000449A8EE08093C20078948091C100806849
:1000D0008093C100E0EFF0E080E40E94C30558E0A7
:1000E000C895802D0E94BD0531965A95C9F704C068
:1000F0001111111F1315081F0E9457058CE00E9453
:10010000C3050E945105ECEFFDE00E944A050E94E4
:100110005505EAE0FEE00E944A05E2E0F0E00E94B8
:100120006C050027A6E2B0E08C9185FB0EF401E09F
:1001300040E0041711F00C946B020E945705E6E1B1
:10014000FEE00E944A05E2E0F0E00E946C0581E0DA
:1001500080931101E1E1F1E0A190BB24ECEFFFEF0E
:10016000AA0CBB1CAA0CBB1CEA0DFB1DACE0B1E049
:1001700094E00E94F7068FEB11E00E946605E2E230
:10018000FEE00E944A05AEEAB4E0E1E1F1E00E943F
:1001900093060E943D05E4E2FEE00E944A05AEEAB5
:1001A000B4E0ECE0F1E00E9487060E943D05E6E243
:1001B000FEE00E944A0580E00E94BD05EAE2FEE002
:1001C0000E944A050027A6E2B0E08C9185FB0EF460
:1001D00001E040E0041711F00C94410184E190E04B
:1001E0000E94F7050027A6E2B0E08C9185FB0EF493
:1001F00001E040E0041711F00C944101A1E1B1E0ED
:10020000BA93AA930E94DF042296E1E1F1E0A19063
:10021000BB24ECEFFFEFAA0CBB1CAA0CBB1CEA0D25
:10022000FB1DACE0B1E094E00E94F7068FEB11E01B
:100230000E946605E2E2FEE00E944A05AEEAB4E0F2
:10024000E1E1F1E00E9493060E943D05E4E2FEE058
:100250000E944A05AEEAB4E0ECE0F1E00E948706B5
:100260000E943D05E6E2FEE00E944A0580E00E9411
:10027000BD05EAE2FEE00E944A0588E592E00E94A0
:10028000F7050027A6E2B0E08C9184FB0EF401E0B4
:1002900040E0041711F00C94690284E190E00E94A0
:1002A000F7050027A6E2B0E08C9184FB0EF401E094
:1002B00040E0041711F00C94690200E010E020E027
:1002C00030E0A8E0B1E00D931D932D933C930E9484
:1002D00051058EE70E94BD05AEEAB4E0E1E1F1E030
:1002E0000E9493060E943D05E6E3FEE00E944A0557
:1002F000E2E0F0E00E946C0580E08093120180E073
:10030000809313018FE714E00E946605AEEAB4E023
:10031000E2E1F1E00E9493060E943D0580E10E9427
:10032000C3058AE0809316010027A6E2B0E08C9115
:1003300085FB0EF401E040E0041711F00C94C601B7
:1003400084E190E00E94F7050027A6E2B0E08C91DE
:1003500085FB0EF401E040E0041711F00C94C60197
:10036000A2E1B1E0BA93AA930E94F3042296AEEA06
:10037000B4E0E2E1F1E00E9493060E943D0580E1D5
:100380000E94C30584EF91E00E94F7050027A6E2D2
:10039000B0E08C9184FB0EF401E040E0041711F012
:1003A0000C94000284E190E00E94F7050027A6E289
:1003B000B0E08C9184FB0EF401E040E0041711F0F2
:1003C0000C94000280911601815080931601A3E1E4
:1003D000B1E08C918F5F8C93A8E0B1E00D911D91FD
:1003E0002D913C91A2E1B1E04C91552766277727EA
:1003F0000E946C06A8E0B1E00D931D932D933D93F0
:1004000000911601003011F00C940A020C943E0287
:100410000C943C0200911301013011F00C943C0249
:10042000A8E0B1E00D911D912D913C914AE050E082
:1004300060E070E00E940606A8E0B1E00D931D9315
:100440002D933D938091130181508093130180E09F
:100450008093120184E10E94C305AEEAB4E0E2E1B8
:10046000F1E00E9493060E943D0580E10E94C305D1
:1004700084EF91E00E94F7050C949401E1E1F1E032
:10048000A190BB24ECEFFFEFAA0CBB1CAA0CBB1C79
:10049000EA0DFB1DA8E0B1E094E07BE70E94E606D0
:1004A0000E9451058CE00E94C305E2E2FEE00E943A
:1004B0004A05AEEAB4E0E1E1F1E00E9493060E9451
:1004C0003D05E6E4FEE00E944A0584EF91E00E94CB
:1004D000F7050C94E200E4E2F0E0A8E1B1E00E944C
:1004E000F4060027A6E2B0E08C9184FB0EF401E054
:1004F00040E0041711F00C94A702A8E1B1E08C9140
:1005000080958C93E4E2F0E0A8E1B1E07BE70E9403
:10051000E3060E945105E6E5FEE00E944A050091CF
:100520001801003011F00C949B02E0E6FEE00E94FE
:100530004A050C949F02E2E6FEE00E944A05E4E6CA
:10054000FEE00E944A05E2E0F0E00E946C0581E0D6
:10055000809317010E9457050E945105A5E0B1E064
:100560000E9463060E94D50480E00E94360583E065
:100570000E94360588E790E00E94F7050E94070573
:10058000A0E1B1E08C9300911001013011F00C94C6
:10059000C9040E940D05A1E1B1E08C930E940D05F4
:1005A000A2E1B1E08C930E940D05A3E1B1E08C9330
:1005B0000E940D05A4E1B1E08C930E940D05A5E118
:1005C000B1E08C93A1E1B1E09C910E94E405A0E12F
:1005D000B1E08C93A0E1B1E00C91112722273327E1
:1005E00040EA56E861E070E00E940606A8E0B1E04B
:1005F0000D931D932D933D93A2E1B1E09C910E9438
:10060000E405A0E1B1E08C93A0E1B1E00C911127E9
:100610002227332748EE53E060E070E00E94060690
:10062000ACE0B1E00D931D932D933D93A8E0B1E0B4
:100630000D911D912D913C91ACE0B1E04D915D91FA
:100640006D917C910E946C06A8E0B1E00D931D9322
:100650002D933D93A3E1B1E09C910E94E405A0E1BC
:10066000B1E08C93A0E1B1E00C9111272227332750
:100670004AE050E060E070E00E940606ACE0B1E0C5
:100680000D931D932D933D93A8E0B1E00D911D9125
:100690002D913C91ACE0B1E04D915D916D917C91DB
:1006A0000E946C06A8E0B1E00D931D932D933D933D
:1006B00094E0A4E1B1E00E942906A8E0B1E00D9128
:1006C0001D912D913C91A4E1B1E04C9155276627F5
:1006D00077270E946C06A8E0B1E00D931D932D933F
:1006E0003D93E7E1F1E0A190BB24ECEFFFEFAA0C12
:1006F000BB1CAA0CBB1CEA0DFB1DACE0B1E094E0F6
:100700000E94F706009118010F3F11F00C949E0310
:10071000ACE0B1E00D911D912D913C91A8E0B1E0CC
:100720004D915D916D917C910E947106A8E0B1E0C0
:100730000D931D932D933D930C94B203A8E0B1E06B
:100740000D911D912D913C91ACE0B1E04D915D91E9
:100750006D917C910E946C06A8E0B1E00D931D9311
:100760002D933D93AEEAB4E0E8E0F1E00E94870605
:100770000E943D05E6E2FEE00E944A0580E00E94FC
:10078000BD050AE00E9445050E945505009115012E
:10079000003011F00C94D203EAE6FEE00E944A0514
:1007A0000C946004013011F00C94DC03E0E7FEE0EF
:1007B0000E944A050C946004023011F00C94E60388
:1007C000E6E7FEE00E944A050C946004033011F055
:1007D0000C94F003ECE7FEE00E944A050C946004E0
:1007E000043011F00C94FA03E2E8FEE00E944A059E
:1007F0000C946004063011F00C940404E8E8FEE068
:100800000E944A050C946004083011F00C940E0408
:10081000EEE8FEE00E944A050C946004003811F0F6
:100820000C941804E4E9FEE00E944A050C9460046C
:10083000013811F00C942204EAE9FEE00E944A0516
:100840000C946004023811F00C942C04E0EAFEE0F1
:100850000E944A050C946004033811F00C9436048D
:10086000E6EAFEE00E944A050C946004083811F0A4
:100870000C944004ECEAFEE00E944A050C946004EB
:100880000A3011F00C944A04E2EBFEE00E944A05A3
:100890000C9460040C3011F00C945404E8EBFEE06E
:1008A0000E944A050C946004AEEAB4E0E5E1F1E090
:1008B0000E9493060E943D05EEEBFEE00E944A0571
:1008C0000027A6E2B0E08C9185FB0EF401E040E049
:1008D000041711F00C94830484E190E00E94F70562
:1008E0000027A6E2B0E08C9185FB0EF401E040E029
:1008F000041711F00C948304A7E1B1E0BA93AA9312
:100900000E94DF04229600911801003011F00C942F
:100910008F04E4ECFEE00E944A050C949304E8EC9A
:10092000FEE00E944A05AEEAB4E0E7E1F1E00E9491
:1009300093060E943D05E4E2FEE00E944A0500277E
:10094000A6E2B0E08C9184FB0EF401E040E00417D5
:1009500011F00C94C30484E190E00E94F705002795
:10096000A6E2B0E08C9184FB0EF401E040E00417B5
:1009700011F00C94C30481E80E9436050E94D5044E
:1009800081E80E9436058AEF90E00E94F7050C94FA
:10099000D104ECECFEE00E944A05E5E0F0E00E94A4
:1009A0006C050C94AC02F894FFCF80E00E943605F1
:1009B00080E00E94360580E00E9436050895A881F7
:1009C000B9818C918F5F8C93A881B9810C9109308A
:1009D00018F011F00C94EE040C94F20481E0A8815C
:1009E000B9818C930895A881B9818C918F5F8C9384
:1009F000A881B9810C91093018F011F00C9402050E
:100A00000C94060580E0A881B9818C9308958091AB
:100A10000701882309F081E0089580910701882368
:100A200009F408950F929F93AF93BF937F938091A2
:100A300007018823E1F3F894809107018A95809358
:100A4000070190910501A0E0B1E0A90F0024B01DBD
:100A50008C919395953009F499279093050178949A
:100A60007F91BF91AF919F910F9008950090C0002A
:100A700005FEFCCF8093C6000895AEEAB4E08D91E8
:100A8000882311F07AD0FBCF089580E276D00A95C2
:100A9000E1F708950E943106802D11F06ED0FACF53
:100AA000089582E070D01ED014C080EC6CC081E04C
:100AB0006AD018D080E867C08FE7213039F08FEB1B
:100AC000223021F08FE8233009F08FEC810F0C9455
:100AD000C30580E858D0089588EE93E088D0319718
:100AE000D9F7089583E0992782C08AEF90E00E94A9
:100AF000F705219A229A239A249A389A3A9A429888
:100B000085E090E00E94F705409829982A982B9A52
:100B10002C9A409AEF93FF93E1E1F1E00E94EB05FC
:100B2000FF91EF91409860D0409AEF93FF93E1E1FD
:100B3000F1E00E94EB05FF91EF91409855D0409A6B
:100B4000EF93FF93E1E1F1E00E94EB05FF91EF915C
:100B500040984AD02C98409AEF93FF93E1E1F1E05E
:100B60000E94EB05FF91EF9140983ED088E20BD0B8
:100B70008EE009D086E007D00895429A829505D08C
:100B800004D032D008954298F9CF859510F42C9A6C
:100B900001C02C98859510F42B9A01C02B9885954F
:100BA00010F42A9A01C02A98859510F4299A01C058
:100BB0002998409AEF93FF93E1E1F1E00E94EB0561
:100BC000FF91EF9140980895892F8F70905110F008
:100BD000865FFCCF08953197F1F70895689462F825
:100BE0000895E89462F8089581E090E000C0EF93E2
:100BF000FF93EE27E82BE92B31F0EDECFAE031978B
:100C0000F1F70197D1F7FF91EF9108950F921F929D
:100C10002F92C801D901489F80014A9F90014B9FA4
:100C2000202C499F100D211D321D5A9F202C589FAA
:100C3000100D211D321D599F200D311D689F200D63
:100C4000311D699F300D789F300D2F901F900F90B0
:100C50000895903029F08C9186959A95E9F78C93B8
:100C60000895C8953196002008957F930F93AF9310
:100C7000BF938F939F938FB78F938091070105E068
:100C8000081B29F49091C6000E94EE0513C0009144
:100C90000601A0E0B1E077279091C600A00FB71F32
:100CA0009C938395809307010395053009F40027F1
:100CB000009306018F918FBF9F918F91BF91AF914C
:100CC0000F917F9118956FB7F894882793E08D93D3
:100CD0009A95E9F76FBF0895040F151F261F371F58
:100CE0000895041B150B260B370B0895000F111FD9
:100CF000221F331F089500951095209530950F5FA2
:100D00001F4F2F4F3F4F0895019110810EC0019149
:100D10001191219130810BC00191108117FF05C005
:100D20003FEF2FEF04C0008111272227332737FF21
:100D300003C0E1DF8DE28D93CF93DF93CF92DF92FB
:100D4000EF92AA24BB24CC24DD24EE2440E2CAE0A6
:100D5000DD2755E093E38881890F87FD9F7083FD30
:100D6000907F891B89935A95A9F7C0DFAA1CBB1CE9
:100D7000CC1CDD1CEE1C4A9551F7E894EFE0FF27F0
:100D800082910ED0EB30E0F71EF068948A2D0CD0E3
:100D900088278D93EF90DF90CF90DF91CF910895CA
:100DA000982F829501D0892F8F70805D26F0803337
:100DB00009F4089568948D930895F999FECFE1BDE3
:100DC000F2BD3196089591E001C092E07B3751F475
:100DD0007FB7F894F2DF8D9180BDFA9AF99A9A95CF
:100DE000C9F77FBF7727089591E001C092E0E5DF62
:100DF000F89A80B58D939A95D1F7089558767274C4
:100E00007220446973706C61790020627920494BCB
:100E1000315A59570000436F6E666967206D6F64E1
:100E200065002300200030302000202020202020DA
:100E30002020202020002047487A4D487A6B487AAD
:100E40006F6F6F2000002073617665642020202082
:100E50002020202000004F5554203D204C4F2000E2
:100E60002B002D002049462020004C53422000003A
:100E70005553422000004357202000004357522082
:100E80000000414D2020000057464D200000464DF7
:100E9000202000004C53424E00005553424E0000AB
:100EA00043572D4E00004357524E0000464D2D4EE5
:100EB0000000444947200000504B54200000556E6C
:100EC0006B6E0000202B0000202D00004572723A4E
:0C0ED00020726164696F204F46463F00AD
:00000001FF
